:0C0000000C942C030C9406050C940000DA
:10000C000C9400000C9400000C9400000C94000064
:10001C000C9400000C9400000C9400000C94470409
:10002C000C9400000C9400000C9400000C944304FD
:10003C000C9400000C94BB0E0C9400000C945B030D
:10004C000C9400000C9400000C9400000C94000024
:10005C000C9400000C9400000C94B3040C9400005D
:10006C000C9400000C9400000C9400000C94000004
:10007C000C9400000C9400000C9400000C940000F4
:10008C001027E80364000A000100001000011000B2
:10009C00010040880000010041434B5F43505F4E1C
:1000AC004F524D414C0D0041434B5F43505F414C0F
:1000BC0041524D0D004D4355205241206C657665E3
:1000CC006C2032206F636375722E0D0A00537461BD
:1000DC007274204D435520696E697469616C2E0DE4
:1000EC000A005374617274204D435520696E697413
:1000FC0069616C2066696E69736865642E0D0A000F
:10010C004D435520696E697469616C204F4B2E0DFF
:10011C000A004D6F64656C3A204D45474136345F9B
:10012C0054797065432E0D0A005665723A2044309E
:10013C002E31322E35302E303038372E50480D0AB5
:10014C0000496E746F204D61696E204C6F6F702E7C
:10015C000D0A0053797374656D204D6178696D7566
:10016C006D2043757272656E74206E6F74206465B9
:10017C0066696E652E0D0A004361626C65206F75B1
:10018C0074206F6620737065632E0D0047756E20AA
:10019C0072656D6F7665206465746563742E0D00F1
:1001AC00435020696E206D61696E206C6F6F7020FA
:1001BC0077697468204F4E5F5245513A2025642C64
:1001CC002025642E25640D00435020696E20636841
:1001DC00617267696E673A2025642C2025642E2590
:1001EC0064203B20636E7443505F4F4B2C20636E36
:1001FC007443505F4E473A2025642C2025640D0033
:10020C004C6F636B6572204F6E2E0D004C6F636BE1
:10021C006572204F66662E0D0052656C6179204F19
:10022C006E2E0D0052656C6179204F66662E0D00A6
:10023C0043757272656E74206C696D69743A202511
:10024C006420410D004D61696E206C6F6F702067EA
:10025C00756E204144433A2025642C2025642E25BC
:10026C00640D00426F6F742073656C662074657347
:10027C00742073746172742E2E2E0D0050726520D2
:10028C006368617267696E672073656C662074655C
:10029C0073742073746172742E2E2E0D004572725D
:1002AC006F72207265636F7665722073656C662061
:1002BC00746573742073746172742E2E2E0D00533A
:1002CC00656C662072656C6179204C2061646320DA
:1002DC0074657374206661696C2E2E2E25640D0A6C
:1002EC000053656C662072656C6179204E206164E8
:1002FC00632074657374206661696C2E2E2E2564E0
:10030C000D0A0053656C66206C65616B6167652036
:10031C0041432074657374206661696C2E0D0A006C
:10032C00436F6E746163746F7220746573742066AE
:10033C0061696C2E0D0A0053656C662074657374CC
:10034C0020726573756C743A2025580D0A004C6543
:10035C00616B61676520444320616C61726D206F35
:10036C006363757220696E2069646C652E0D004C98
:10037C0065616B61676520444320616C61726D201F
:10038C006F6363757220696E206368617267696E52
:10039C00672E0D004C65616B616765207265747228
:1003AC00792E2E2E25642E0D004C65616B616765D0
:1003BC0020414320616C61726D206F636375722004
:1003CC00696E2069646C652E0D004C65616B61670C
:1003DC006520414320616C61726D206F636375729F
:1003EC0020696E206368617267696E672E0D00006C
:1003FC0041502073656374696F6E20636865636B2D
:10040C0073756D2063616C2C20666C6173683A2087
:10041C00253034582C20253034582E0D0A00426FCC
:10042C006F742073656374696F6E20636865636BAA
:10043C0073756D2C20666C6173683A2025303458C6
:10044C002C20253034582E0D0A0057617463682017
:10045C00646F67207465737420706173732E0D0A5A
:10046C0000576174636820646F672074657374202F
:10047C006661696C2E0D0A004350552073746174CB
:10048C007573207465737420706173732E0D0A007C
:10049C0043505520737461747573207465737420A4
:1004AC006661696C2E0D0A005372616D2074657360
:1004BC007420706173732E0D0A005372616D207479
:1004CC00657374206661696C2E0D0A0054696D6544
:1004DC007230207465737420706173732E0D0A0072
:1004EC0054696D6572302074657374206661696C33
:1004FC002E0D0A0054696D65723120746573742079
:10050C00706173732E0D0A0054696D65723120741D
:10051C00657374206661696C2E0D0A0054696D65F3
:10052C007232207465737420706173732E0D0A001F
:10053C0054696D6572322074657374206661696CE0
:10054C002E0D0A0054696D65723320746573742026
:10055C00706173732E0D0A0054696D6572332074CB
:10056C00657374206661696C2E0D0A00496E7465A2
:10057C007272757074207465737420706173732E4D
:10058C000D0A00496E74657272757074207465730F
:10059C0074206661696C2E0D0A00466C61736820CC
:1005AC007465737420706173732E0D0A00466C6150
:1005BC0073682074657374206661696C2E0D0A0073
:1005CC00414443207465737420706173732E0D0A5B
:1005DC00004144432074657374206661696C2E0D70
:1005EC000A004750494F207465737420706173730F
:1005FC002E0D0A004750494F2074657374206661B4
:10060C00696C2E0D0A00436C6F636B2074657374F8
:10061C0020706173732E0D0A00436C6F636B207432
:10062C00657374206661696C2E0D0A0001002D4EF5
:10063C00414E00494E460000040002009E0001009D
:10064C005206A20001005A0638060000F894EE2764
:10065C00ECBBF1E0F5BFE5BFE0936C008DE0A2E0F0
:10066C00BB27ED938A95E9F780E090E1A0E0B1E03B
:10067C00ED930197E9F7E4E4F6E085919591009705
:10068C0061F0A591B59105901590BF01F001059011
:10069C000D920197E1F7FB01F0CFEFEFEDBFE0E139
:1006AC00EEBFC0E0D5E00C9416050E946D101A93B5
:1006BC000A931BB10CB1E12FEC7109F0DBC020FCEB
:1006CC00BCC0033411F434FE01C006C0689420F899
:1006DC00E0E0E0935706B0C0023071F4E2E0F0E0E5
:1006EC00E093F805F093F905E0E0E093490668948F
:1006FC0034F8E0934A06A0C0033009F073C0E091CF
:10070C004906F0E03197E75FF94FE081F0E0A09106
:10071C00F805B091F905AE1BBF0BEA17FB0709F002
:10072C0060C0A0910906A03E91F4E0910A06E03069
:10073C0029F4E89453F8E4EAF0E004C0689453F820
:10074C00E3EBF0E0FA93EA930E947B104AC0E89442
:10075C0053F8E0910906E09307060E94801041F4DB
:10076C00A0910706A03418F0EFE3E093070637C01A
:10077C00E230A0E0FA0741F4A0910706A13218F08C
:10078C00E0E2E09307062BC0E330A0E0FA0741F467
:10079C00A0910706A53118F0E4E1E09307061FC00D
:1007AC00E430A0E0FA0741F4A0910706A13118F05B
:1007BC00E0E1E093070613C0E530A0E0FA0741F44E
:1007CC00A0910706AE3018F0EDE0E093070607C0E5
:1007DC00A0910706AE3018F0EDE0E0930706DD9926
:1007EC00ADD328C034FE1EC0E0914906F0E0E75FAF
:1007FC00F94F0083E02FF0E0A091F805B091F905D6
:10080C00EA0FFB1FE093F805F093F905E091490618
:10081C00EF5FE0934906A0914906A03210F0E894EE
:10082C0034F80AC0A0914A06AF5FA0934A06A150C3
:10083C00A13210F0E89434F81DC00B3721F4E0918C
:10084C005706EF5F0FC0033D21F4E0915706EF5FB1
:10085C0009C0013121F4E0915706EF5F03C0E89421
:10086C0020F8E0E0E0935706A0915706A33010F073
:10087C000E949A0E0991199162C00E946D10A4D524
:10088C005EC00E946D10E4E9E4BDF60131966F0183
:10089C00D601EAE0F0E00E948712309721F40024A0
:1008AC000C140D0408F019C026FCA8950E94C10E6A
:1008BC00E03049F4E2E0E0935106E1ECF0E00E9414
:1008CC0088100E949A0E22FCEED443FE02C044FE15
:1008DC0001C003C096D70E94730DD6010E948B10E5
:1008EC00D601E4EFF1E00E948712309721F4002446
:1008FC000C140D0408F002C0689455F8D601E8EE0B
:10090C00F3E00E948712D601ECEDF5E00E9487120D
:10091C00309721F400240C140D0408F009C0A091A8
:10092C005006AF3F28F4E0915006EF5FE09350067D
:10093C00E0EDF7E0CE16DF0610F0CC24DD24E991D3
:10094C00EFBFF991E991B991A99199918991799117
:10095C006991F990199009901895AA93BA93EA9312
:10096C00FA93EFB7EA93E0918000F0E0E093FA0598
:10097C00F093FB05E0918100FE2FE0E0A091FA05D9
:10098C00B091FB05EA2BFB2BE093FA05F093FB05EA
:10099C00E0918A00E07451F00E949010E093FE0503
:1009AC00F093FF05EEB5EF7BEEBD23C0A091FE05E5
:1009BC00B091FF050E949010EA1BFB0BE093000620
:1009CC00F0930106A091FC05B091FD050E949010DA
:1009DC00EA1BFB0BE0930206F09303060E949010B7
:1009EC00E093FC05F093FD05E0918A00E064E09350
:1009FC008A00E991EFBFF991E991B991A991189504
:100A0C001895AA93E881E064E7B985E28A95F1F735
:100A1C00369A349BFECF349AE4B1F5B12196089501
:100A2C000E949510E0916300E17021F4A8EBBBE00B
:100A3C000E944414E9EDF0E00E9488100E94190E07
:100A4C00EEEEF0E00E948810E0916300E17021F47A
:100A5C00A8E8B3E10E9444140E949C10AB9833FEAA
:100A6C0010C0ECE0F1E00E9488100E94A210EEE1B0
:100A7C00F1E00E9488100E94A210E5E3F1E00E94D0
:100A8C008810A1E003D3E0934D06689443F8EDE49D
:100A9C00F1E00E9488100E94A61030FC02C00E9457
:100AAC00AE10E0916300E17081F4A0915306B09117
:100ABC005406A93EE3E0BE0718F0E89425F804C0FC
:100ACC00A3E5B6E00E94B71007C0E0E0E093530640
:100ADC00E0935406689425F825FC36C0E0E0E093DA
:100AEC005306E0935406E89432F8A0910205B091B5
:100AFC000305109711F453FE0DC0A8D30E94A61243
:100B0C0020F4E3EBF0E00E948810A0E0B0E080E07D
:100B1C0090E009C09BD3309721F4E4EAF0E00E9406
:100B2C0088100E94BD1074D3E89427F830F831F87F
:100B3C00E0E0E093F405E093F505E0E2E0930706CE
:100B4C000E949C10A0E074C1E0910806E03009F00E
:100B5C006AC130FC35C1E89453F80E94C2100E945F
:100B6C00AE1033FE02C0689445F80E94C510EE38F2
:100B7C00A2E0FA0730F00E94CA10A033E3E0BE07EF
:100B8C0068F00E94C510E939A1E0FA0730F00E9424
:100B9C00CA10AB33E2E0BE0708F011C1A2E076D276
:100BAC00E0934E0631FC04C0A0914E06A03009F033
:100BBC0006C10E94CF100E94A61033FE02C068949A
:100BCC0052F821FED6C00E94D710E531A1E0FA07F9
:100BDC0030F00E94DC10AF33E1E0BE0708F027C014
:100BEC000E94E11019F40E94E81020C0E230A0E04D
:100BFC00FA0719F40E94F11019C0E330A0E0FA07CB
:100C0C0019F40E94FA1012C0E430A0E0FA0719F4AB
:100C1C000E9403110BC0E530A0E0FA0719F40E9402
:100C2C000C1104C00E94C2100E941511A1C00E9498
:100C3C00D710E03BA1E0FA0730F00E94DC10AA3E8E
:100C4C00E1E0BE0708F027C00E94E11019F40E94F1
:100C5C00E81020C0E230A0E0FA0719F40E94F1106D
:100C6C0019C0E330A0E0FA0719F40E94FA1012C080
:100C7C00E430A0E0FA0719F40E9403110BC0E53030
:100C8C00A0E0FA0719F40E940C1104C00E94C210D3
:100C9C000E9415116DC00E94D710E337A2E0FA072D
:100CAC0030F00E94DC10A73BE2E0BE0708F027C042
:100CBC000E94E11019F40E94E81020C0E230A0E07C
:100CCC00FA0719F40E94F11019C0E330A0E0FA07FA
:100CDC0019F40E94FA1012C0E430A0E0FA0719F4DB
:100CEC000E9403110BC0E530A0E0FA0719F40E9432
:100CFC000C1104C00E94C2100E94151139C00E9430
:100D0C00D710EA3CA2E0FA0718F00E941A1108F07A
:100D1C0027C00E94E11019F40E94E81020C0E230B4
:100D2C00A0E0FA0719F40E94F11019C0E330A0E01A
:100D3C00FA0719F40E94FA1012C0E430A0E0FA0786
:100D4C0019F40E9403110BC0E530A0E0FA0719F466
:100D5C000E940C1104C00E94C2100E94151108C000
:100D6C000E94C210E89430F8E4E8F1E00E94881088
:100D7C0026C00E94801019F40E94E81020C0E230B6
:100D8C00A0E0FA0719F40E94F11019C0E330A0E0BA
:100D9C00FA0719F40E94FA1012C0E430A0E0FA0726
:100DAC0019F40E9403110BC0E530A0E0FA0719F406
:100DBC000E940C1104C00E94C2100E94151118C090
:100DCC0053FE0EC043D20E94A61248F4A0E0B0E03D
:100DDC0080E090E01DD2E3EBF0E00E94881008C0A8
:100DEC0035D2309729F4AAD0E4EAF0E00E948810BA
:100DFC000E94CA10A335E3E0BE0790F033FE04C096
:100E0C000E941F11E03009F006C00E942511E8E98C
:100E1C00F1E00E9488100E941F110E94C21002C0B3
:100E2C000E949C1006C0A0910806A13011F4A1E00C
:100E3C0016D245FE0EC00E942511ECEAF1E00E948C
:100E4C0029110E9469118CE00E9425102E96E894BD
:100E5C0045F846FE16C00E942511E4EDF1E00E9413
:100E6C0029110E946911E09105060E946E11E09112
:100E7C0006060E946E1184E10E9425106696E89485
:100E8C0046F847FE0FC00E942511C99B03C0ECE039
:100E9C00F2E002C0E8E1F2E0FA93EA930E947B10E0
:100EAC00E89447F850FE0FC00E942511DD9B03C04B
:100EBC00E5E2F2E002C0E0E3F2E0FA93EA930E948A
:100ECC007B10E89450F851FE0EC00E942511ECE303
:100EDC00F2E0FA93EA93E09107060E946E110E94E9
:100EEC007411E89451F852FE27C00E942511E1E5D7
:100EFC00F2E0FA93EA930E94D7100E9469110E94C3
:100F0C0079110E94D712FF2766277727FF276627BC
:100F1C0077270E949C120E9479110E94BD100E949A
:100F2C008D11DF010E948B100E9469118CE00E94D0
:100F3C0025102E96E89452F8B0CDFFCF21FE85C037
:100F4C000E94941130F00E94DC10AF33E1E0BE0738
:100F5C0008F01FC0E0910706E73020F0A0910706CB
:100F6C00A43308F005C00E9499110E94A3110DC072
:100F7C00E0910706E43320F0A0910706A13508F0B4
:100F8C0007C00E9499110E94AA11DF01CB0140D128
:100F9C005BC00E94D710E03BA1E0FA0730F00E9442
:100FAC00DC10AA3EE1E0BE0708F011C0A0910706D4
:100FBC00A13238F40E9499110E94A311DF01CB01D8
:100FCC0004C0A5E5B5E585E592E422D13DC00E94BB
:100FDC00D710E337A2E0FA0730F00E94DC10A73BF1
:100FEC00E2E0BE0708F011C0A0910706A13138F469
:100FFC000E9499110E94A311DF01CB0104C0A5E549
:10100C00B5E585ED91E404D11FC00E94D710EA3CF0
:10101C00A2E0FA0718F00E941A1108F011C0A09172
:10102C000706AE3038F40E9499110E94A311DF011B
:10103C00CB0104C0A5E5B5E58DEA91E4E9D004C087
:10104C000E94C210E89430F81EC0E0910706E73009
:10105C0020F0A0910706A43308F005C00E94991156
:10106C000E94A3110DC0E0910706E43320F0A0917B
:10107C000706A13508F007C00E9499110E94AA1119
:10108C00DF01CB01C5D0689451F80895AA930E9452
:10109C004A1210E0689444F833FE1CC00E94A2105F
:1010AC00EC81F0E0E130A0E0FA0719F4EFE6F2E0B1
:1010BC000DC0E230A0E0FA0719F4E8E8F2E006C04F
:1010CC00E330A0E0FA0731F4E9EAF2E0FA93EA93AC
:1010DC000E947B10DF980E942511DF9AAAE0B0E0F5
:1010EC000E944414DF980E9425110E94B711D8F079
:1010FC001460DA9A0E94A210DA980E94A210DA9A6E
:10110C000E94A210DA980E94A210DA9A0E94A210F1
:10111C00DA980E94A21033FE06C0EBECF2E00E94BB
:10112C00CA110E9474111C980E9425111C9AAAE0E5
:10113C00B0E00E9444141C980E9425110E94B71123
:10114C00D8F01860DA9A0E94A210DA980E94A210C5
:10115C00DA9A0E94A210DA980E94A210DA9A0E94DF
:10116C00A210DA980E94A21033FE06C0EDEEF2E057
:10117C000E94CA110E94741140FE1BC0E0916200D3
:10118C00E068E0936200A8E5B2E00E9444149A99EA
:10119C0007C0116033FE04C0EFE0F3E00E9488103A
:1011AC00E0916200EF77E0936200A0EBB4E00E9464
:1011BC00441437FE1BC0869B19C01061DA9A0E943A
:1011CC00A210DA980E94A210DA9A0E94A210DA9861
:1011DC000E94A210DA9A0E94A210DA980E94A21021
:1011EC0033FE04C0ECE2F3E00E94881033FE09C029
:1011FC00E3E4F3E0FA93EA93E12F0E946E110E946C
:10120C007411E89444F8E12F0E9451122596089528
:10121C000E94A1120E94D0110E948D11EF2FF0E0BC
:10122C00EBBD0E94D0110E9492130E94D712EABD0E
:10123C000E949712E0E0F0E068EC72E40E94241443
:10124C0010F4A1E001C0A0E0E2D48DC5EBB5FE2FF7
:10125C00E0E0DF01EAB5F0E0EA2BFB2B0895AA935E
:10126C00E881E03079F033FE02C0DD9B01C002C0A2
:10127C00689450F8DD9AE0916500E260E0936500B7
:10128C0068940EC033FE02C0DD9901C002C06894A0
:10129C0050F8DD98E0916500ED7FE0936500E894EF
:1012AC0032F80C94DD0E0E94D711AF3FE0E0BE0780
:1012BC0020F4A4E0B5E00E94B71032FE46C00E94B4
:1012CC00941118F00E941A1108F03EC0C99B04C07A
:1012DC00A0914B06A33060F523FE20C00E94D711CD
:1012EC00549718F4DB98DC9A18C0E0910405F0913F
:1012FC000505759720F00E94D711989708F002C049
:10130C00DC980BC00E94D711A436E0E0BE0728F091
:10131C00E0E0E0930405E093050501C0DB9A33FEA1
:10132C0004C0A0914B06A03009F002C0689447F8A5
:10133C00A0914B06A33028F4E0914B06EF5FE093AD
:10134C004B06E0E0E0934C063EC0C99904C0A09166
:10135C004C06A33060F523FE20C00E94D711549791
:10136C0018F4DC98DB9A18C0E0910405F09105059F
:10137C00759720F00E94D711989708F002C0DB985F
:10138C000BC00E94D711A436E0E0BE0728F0E0E0C5
:10139C00E0930405E093050501C0DB9833FE04C01F
:1013AC00A0914C06A03009F002C0689447F8A091B7
:1013BC004C06A33028F4E0914C06EF5FE0934C060A
:1013CC00E0E0E0934B06089530FE04C0809B02C021
:1013DC009F9901C015C2A0E014DB5F010E94CF10E1
:1013EC00E0910805F0E03F970CF06DC0AEE2B3E081
:1013FC00AA15BB0528F4E7E1F4E0AE16BF0608F029
:10140C000CC0E0910905AEE0B5E00E94DC11E09162
:10141C000905EF5FE093090550C0A5E4B2E0AA15F9
:10142C00BB0528F4EEE2F3E0AE16BF0608F00CC0E4
:10143C00AEE2B5E0E0910A050E94DC11E0910A05EC
:10144C00EF5FE0930A0539C0ADE5B1E0AA15BB0525
:10145C0028F4E5E4F2E0AE16BF0608F00CC0AEE4EA
:10146C00B5E0E0910B050E94DC11E0910B05EF5FFC
:10147C00E0930B0522C0A4E7B0E0AA15BB0528F445
:10148C00EDE5F1E0AE16BF0608F00CC0AEE6B5E037
:10149C00E0910C050E94DC11E0910C05EF5FE093EC
:1014AC000C050BC0AEE8B5E0E0910D050E94DC1117
:1014BC00E0910D05EF5FE0930D05E0910805EF5FFE
:1014CC00E093080575C0E0910905E0930605E0E09E
:1014DC00E0930705E1E0F0E04F01E5E0F0E08E1667
:1014EC009F0690F40E94E411AC91E0910605EA1776
:1014FC0038F40E94E411EC91E09306058092070504
:10150C00F40131964F01E9CFE89424F8882499240A
:10151C00E5E0F0E08E169F06A8F4E0910705D401F3
:10152C00F0E0EA17FB0739F00E94E411AC910E943D
:10153C00E911EA1709F002C0689424F8F401319615
:10154C004F01E6CF24FC27C0AA24BB24882499246D
:10155C000E94E911D401F0E0AE17BF0788F4E091C6
:10156C000705F0E0EE0FFF1F0E946612E25FFA4FD4
:10157C00DF01F4010E94F011F40131964F01E8CF24
:10158C000E94E911F0E0D5010E947412B696E09326
:10159C00F005F093F105E0E0E0930805E093090510
:1015AC00E0930A05E0930B05E0930C05E0930D0521
:1015BC0054FE38C0E0910406AEEAB5E0F0E0EE0F60
:1015CC00FF1FEA0FFB1FFF93EF93A1E01ADAAF9115
:1015DC00BF91ED93FC93E0910406F0E07F9724F427
:1015EC00E0910406EF5F01C0E0E0E0930406AA245A
:1015FC00BB2488249924E0E2F0E08E169F0648F480
:10160C00F401AEEAB5E00E94F011F40131964F01FD
:10161C00F2CFD501E0E2F0E00E947412E093EE0507
:10162C00F093EF0533FE18C0A0910005B0910105B1
:10163C00A938E3E1BE0778F4A091F205B091F30567
:10164C000E94C510EA1BFB0BDF010E944A10E73415
:10165C00A0E0FA0708F001C00EC0689446F8E0E07C
:10166C00E0930005E09301050E94C510E093F2059C
:10167C00F093F30504C0A0E0B5E00E94B71040FE63
:10168C0031C0A0910506A03218F0E8E9F1E002C0E3
:10169C00ECE7F1E0DF010E94C510AE17BF0770F454
:1016AC00A0910506A03218F0EBE3F2E002C0E6E2EE
:1016BC00F2E00E94CA10AE17BF0708F011C025FE59
:1016CC000FC00E94F91160F427FC0AC0A0915506C6
:1016DC00A13031F09A9904C0999902C0E1E001C09F
:1016EC00E0E028C0A0910506A03218F0E8E9F1E08E
:1016FC0002C0ECE7F1E0DF010E94C510AE17BF0796
:10170C0070F4A0910506A03218F0EBE3F2E002C0F1
:10171C00E6E2F2E00E94CA10AE17BF0708F009C05B
:10172C0025FE07C00E94F91120F427FC02C0E1E05D
:10173C0001C0E0E0E03001F1A0910506A03228F4F0
:10174C00E0910506EF5FE0930506A0910506A03237
:10175C0090F0E0E0E0930606A1E081DD0E94CA1063
:10176C00A335E3E0BE0728F00E941F110E94C210AF
:10177C0002C00E949C1044C00E94DC10E091F6054F
:10178C00F091F705EA1BFB0BDF010E944A103F9713
:10179C00B8F5A0910606A03228F4E0910606EF5F9A
:1017AC00E093060640FE10C0A0910606A03250F44D
:1017BC00A0915506A13031F09A9904C0999902C0B4
:1017CC00E0E001C0E1E010C0A0910606A03220F4D8
:1017DC00A0915506A13009F406C00E941F11E030FB
:1017EC0011F4E0E001C0E1E0E03051F00E94F911A9
:1017FC0010F0689427F8E0E0E0930506A0E02FDDF8
:10180C0008950E94011270F1E0E0E0934F06E0931E
:10181C005506E0914E06EB7F0E940612E77F0E9470
:10182C000612EE7F0E940612ED7FE0934E060E9498
:10183C000912EF7D0E940E120E940912EF7B0E948A
:10184C000E12E0910305E77FE0930305E091560645
:10185C00E03041F40E940912E77F0E941312EB7FE3
:10186C000E940E1254FE0DC027FE04C00E940912E5
:10187C00E26003C00E940912ED7FE0930205F09331
:10188C00030540FE4EC0999B02C09A9B01C029C023
:10189C00E0910205E470B1F4E0E0E093500633FE11
:1018AC0004C0E0915506E03009F00CC00E94011212
:1018BC0018F0EAE5F3E002C0EBE7F3E0FA93EA9301
:1018CC000E947B10E1E0E09355060E94011210F09B
:1018DC00E1E001C0E0E0E09356060E940912E460EA
:1018EC001CC0A0915006AF3240F0E0915506E0309C
:1018FC0021F0A0914F06A13008F013C00E941512E0
:10190C0033FE04C00E941E120E947411A3E0BEDBC1
:10191C00E03039F40E942512E77FE0930205F09342
:10192C00030540FE52C09A9B02C0999905C09A9B30
:10193C0002C0999B01C029C0E0910205E870B1F486
:10194C00E0E0E093500633FE04C0E0915506E03031
:10195C0009F00CC00E94011218F0E5EBF3E002C094
:10196C00E6EDF3E0FA93EA930E947B10E1E0E0935A
:10197C0055060E94011210F0E1E001C0E0E0E09396
:10198C0056060E940912E8601CC0A0915006AF32A6
:10199C0040F0E0915506E03021F0A0914F06A130C7
:1019AC0008F013C00E94151233FE04C00E941E12D0
:1019BC000E947411A3E06ADBE03039F40E94251216
:1019CC00E77FE0930205F0930305E0914D06E1708B
:1019DC0061F4E0914D06E27041F4E0914E06E17045
:1019EC0021F4E0914E06E27029F0E0910305E860E5
:1019FC00E093030522FE1CC032FE06C0C99904C048
:101A0C00A0914B06A43048F432FC06C0C99B04C01C
:101A1C00A0914C06A43008F404C00E940912E160A5
:101A2C0003C00E940912EE7FE0930205F0930305B8
:101A3C0036FE22C00E94941118F00E941A1108F070
:101A4C000EC00B9B04C00E940912E06103C00E94EF
:101A5C000912EF7EE0930205F09303050DC00B997C
:101A6C0004C00E940912E06103C00E940912EF7EBB
:101A7C00E0930205F0930305E0914D06E07121F42B
:101A8C00E0914E06E07129F0E0910305E460E093EB
:101A9C000305E0914D06E47021F4E0914E06E470EC
:101AAC0029F00E940912E0620E940E12E0914D068C
:101ABC00E87021F4E0914E06E87029F00E940912BA
:101ACC00E0640E940E12A0915106A13029F4E0911D
:101ADC000305E061E093030508950E940912E1708B
:101AEC00F0700E94A61210F4AB9A8DC00E940912DD
:101AFC00E270F0700E94A61218F4AB98AC9A84C0F5
:101B0C000E940912E470F0700E94A61218F4AB9AAD
:101B1C00AC9A7AC00E940912E870F0700E94A6126A
:101B2C0020F4AB98AC98AD9A70C00E940912E07189
:101B3C00F0700E94A61220F4AB9AAC98AD9A65C0D6
:101B4C000E940912E072F0700E94A61220F4AB9869
:101B5C00AC9AAD9A5AC00E940912E074F0700E94BF
:101B6C00A61220F4AB9AAC9AAD9A4FC00E940912FF
:101B7C00E078F0700E94A61228F4AB98AC98AD985F
:101B8C00AE9A44C00E940912E070F1700E94A61235
:101B9C0028F4AB9AAC98AD98AE9A38C00E94091252
:101BAC00E070F2700E94A61228F4AB98AC9AAD9833
:101BBC00AE9A2CC00E940912E070F4700E94A6121A
:101BCC0028F4AB9AAC9AAD98AE9A20C00E94091238
:101BDC00E070F8700E94A61228F4AB98AC98AD9AFD
:101BEC00AE9A14C00E940912E070F0710E94A61205
:101BFC0028F4AB9AAC98AD9AAE9A08C00E94091220
:101C0C00309721F4AB98AC98AD98AE980895AA9300
:101C1C00E881E03019F0E7B7E46002C0E7B7EB7F8A
:101C2C00E7BF0C94DD0EECEFEABBE0E0EBBBE0E3CE
:101C3C00E7BBE0E0E8BBE8E7E4BBE0E0E5BBE2E201
:101C4C00E1BBE0E0E2BBE0E1E2B9E0E0E3B9E0EC0B
:101C5C00E0936100E0E0E09362000E949510E0E008
:101C6C00E0BFE3BFE2BFE1BFE2E8EFBDE9E1EEBDFB
:101C7C00E0E0EDBDECBDEBE2E7BDE2E3E6BDEBE29F
:101C8C00EBBDE2E3EABDE0E0E9BDE8BDE09379003D
:101C9C00E0937800E5E0E5BDE4E9E4BDE0E0E3BD18
:101CAC00E0938B00E1ECE0938A00E0E0E0938900A4
:101CBC00E0938800E0938100E0938000E09387003C
:101CCC00E0938600E0938500E0938400E09383002A
:101CDC00E0938200E0E4E7BFE0E2E0937D00E0E027
:101CEC00E0936A00EABFE9BFEBB9E8E9EAB9E6E0DC
:101CFC00E0939500E5E0F0E03F017092900069B848
:101D0C00E0E0E0939A00E0E8E8B9E0E4E7B9E7E85E
:101D1C00E6B9E0E0E0BDEDB9E0937400EFE1E1BDC0
:101D2C00EFE0E1BD789408950E944A1200E010E0C3
:101D3C0020E030E0E0E0E1BDE89426F800E010E0BF
:101D4C000F3FEFEF1E0768F420E030E02F3FEFEF7E
:101D5C003E0720F400002F5F3F4FF8CF0F5F1F4F5F
:101D6C00EFCF0E94511224960895EA93E1E0E0939C
:101D7C005906E99118951A930A930DB71127EEB7E6
:101D8C00FE2FE0E08F010130EDE01E0720F0003067
:101D9C00E1E11E0708F002C0E1E001C0E0E00991BA
:101DAC0019910895AA935D9BFECFE881ECB9219619
:101DBC000895BA93AA93AA81F5DFA881B9810E94EC
:101DCC00B71023960895BA93AA9326970E944812A7
:101DDC0010E0AC85BD85E0E0F0E0ED93FC93EA8982
:101DEC00FB893196EA8BFB8B3197E4912E2FE030F7
:101DFC0009F41DC1E12FE03039F4253211F411E062
:101E0C0002C00E942B1212C1E130A9F4253219F440
:101E1C000E942B120AC112E040E000E02D3211F4B6
:101E2C0001E004C12B3211F44BE200C1203211F459
:101E3C0040E2FCC002C0E23039F450E013E0203341
:101E4C0011F40068F3C003C0E33009F0EFC0203395
:101E5C0010F02A3308F007C0AAE05A9F502DE22F49
:101E6C00E0535E0FE3C0E22FE33649F40E943212D6
:101E7C00E889F989A481AA930E943812D6C0E33765
:101E8C0041F40E9432120E943E120E9454101E2FE6
:101E9C000AC0E03761F40E9432120E943E120E9486
:101EAC0060101E2F086002600F7730E03CC0E436F3
:101EBC0011F0E93611F4046002C0E53731F4ECE8B6
:101ECC00F0E0EE83FF8315E00CC0E83511F40860F8
:101EDC0003C0E83709F0A9C0E6E9F0E0EE83FF8320
:101EEC0014E002FF17C00E943212A889B989149617
:101EFC00ED91FD91EA87FB87AB85AA232AF40E941A
:101F0C005A12EA87FB874DE2403011F01F5F01C087
:101F1C000B7F09C00E943212A889B98914960E94BD
:101F2C008A12EA87FB8700FD11C0151778F407FFAA
:101F3C0008C002FF04C00B7F242F115001C020E306
:101F4C0001C020E20E942B125150EFCF312F01FF24
:101F5C0017C03030A1F003FF06C0EE81FF81259140
:101F6C00EE83FF8305C0AE81BF812D91AE83BF830D
:101F7C000E942B12503009F051503150EACF4BC017
:101F8C0020E3EE81FF810E948E12E887F987EE81B3
:101F9C00FF813296EE83FF83E885F985AA85BB85A0
:101FAC00AE17BF0750F02F5FA885B985EA85FB8572
:101FBC00EA1BFB0BEA87FB87EFCF2A3328F003FFE2
:101FCC0002C0295F01C0295D04FD1AC0213320F431
:101FDC00A885B985119709F409C0531710F000FFB3
:101FEC0001C013C020E207FF0BC020E3006102FF19
:101FFC0007C00B7F4A930E943812503009F05150A1
:10200C000E942B12503009F051503150A885B985DF
:10201C00129708F0B5CF00FF08C0503031F0515086
:10202C00E0E2EA930E943812F8CF10E0D8CEAC85EB
:10203C00BD85ED91FD910E944F1264960895FF921B
:10204C00F82E26971A930A93DE0114960E945612C4
:10205C008D01E0E0EC83ED83EE83EF83DE011896D7
:10206C000E945612ED91FD91FA93EA931A930A93FA
:10207C00EFEDFEE0FA93EA93DE011896A4DE1981E7
:10208C0008812896FF900895BA93AA93E991F99143
:10209C0030971AF4E095F09531960895BA93AA9377
:1020AC00A991B991EE27FF276D91662311F0319616
:1020BC00FBCF0895BA93AA93AA27BB27E991F9916C
:1020CC000590002011F01196FBCFFD0108950A92A6
:1020DC001A92FA926A937A938A939A93AA93BA93DE
:1020EC00EA93FA93EFB7EA93089580E00E942510E3
:1020FC0022960895E1E0E0935206F0E0E130A0E092
:10210C00FA070895FA93EA93F0CFE4E6F0E00E9420
:10211C0087120895E091FA05F091FB050895E6E029
:10212C00E0936400E0E0E09365000895E0916500C1
:10213C00EB7FE09365000895A8ECB0E00C94441498
:10214C00A2E00E940705E093F605F093F7050895C9
:10215C00A0E00E940705B696E093F005F093F10518
:10216C000895ED91FD913196FE93EE930895A0E0C4
:10217C00B0E088EC92E40895FADF0C940E09E0913B
:10218C00F005F091F1050895A091F005B091F105DD
:10219C000895A2E00E940705E093F405F093F5057D
:1021AC000895E091F405F091F5050895A091F405DA
:1021BC00B091F5050895E0915206F0E0E130A0E011
:1021CC00FA070895A6E6B6E682EB92E40E940E09A1
:1021DC00689430F80895A5E5B5E585E592E40E948C
:1021EC000E09689430F80895A5E5B5E585E092E40C
:1021FC000E940E09689430F80895A5E5B5E585EDC3
:10220C0091E40E940E09689430F80895A5E5B5E5AF
:10221C008DEA91E40E940E09689430F80895E894D0
:10222C0030F8EFE5F1E06ECFC1DFAD30E3E0BE0793
:10223C000895E0916500E460E09365000895A4E6DC
:10224C00B0E00C944414FA93EA9399DF662777274D
:10225C000E949C1294DF662777270E941013DF01DF
:10226C00CB01E0E0F0E060E874E40E94E013A3E34B
:10227C00B3E383E591E40E9492130E94D712FF27E7
:10228C0066277727FF27662777270E949C1277DF20
:10229C00662777270E941013DF01CB01E0E0F0E006
:1022AC0060E874E40E94E013A3E3B3E383E591E4F4
:1022BC000E9492135CDF0E9492130E94D712662731
:1022CC007727DF0122CF662777270E949C1208957B
:1022DC00FF27662777270E949C12089584E00E94AE
:1022EC002510269608955DDF662777270E94101328
:1022FC00A3E3B3E383E590E40E949213DF01CB01E7
:10230C00E0E0F0E060E874E40E94E01308950E94BD
:10231C0092130E94D71266277727089542DFE53182
:10232C00A1E0FA070895E0910706F0E00E946F1211
:10233C000E941013DF01CB010895EAE9F9E969E184
:10234C007FE30E94E0130895E0E0F0E060E270E4C7
:10235C000E94E013A0E0B0E080E892E40E944313F6
:10236C00089520E030E0A4E00E9407052E0F3F1FE7
:10237C00A4E00E9407052E0F3F1FF901F695E79583
:10238C00EC39A0E0FA070895FA93EA93F901F6956F
:10239C00E79599CF0E949212A6EFB8E28DED92E4E8
:1023AC000895A0910405B09105050895F0E0EE0F95
:1023BC00FF1FEA0FFB1FA082B1820895A9E0B5E0D0
:1023CC00A80DB91D0895E0910705F0E0E75FFA4FFD
:1023DC00E0810895EE0FFF1FAE0FBF1F0E948A12FF
:1023EC00AE0EBF1E0895A091EE05B091EF05A83B6F
:1023FC00EBE0BE070895C8DEA133E3E0BE07089505
:10240C00E0934E060895E0910205F09103050895BE
:10241C00E0930205F09303050895FADFF4CFE0E0B2
:10242C00E0935006E0914F06EF5FE0934F0608955E
:10243C00E0EAF3E0FA93EA93E0914F0649CFE0E04B
:10244C00E0935506E0DFEB7FE8CF2A93AD85BE85A0
:10245C00EF85F88909950895E889F9893497E88B0F
:10246C00F98B0895AD85BE85EF85F889099508959A
:10247C00A889B9891496ED91FD91EE83FF83AE8105
:10248C00BF8108955A934A933A932A931A930A93C5
:10249C0008955D814C813B812A81198108810895C1
:1024AC000024AF0DB01D0895F195E195F04008950D
:1024BC00F09560957095E195FF4F6F4F7F4F0895A4
:1024CC00EE0FFF1FEE0FFF1FEE0FFF1FEE0FFF1F94
:1024DC0008956F2F660F660B762F08950024112434
:1024EC0090E1AA0FBB1F001C111C0E1A1F0A18F436
:1024FC000E0E1F1E01C0A1609A9599F7FD01D00127
:10250C000895ECDFFD010895ED91FC91119708956C
:10251C000590F491E02D0895E881F9816A817B8121
:10252C000895A881B9818A819B8108957A936A93D1
:10253C00FA93EA9308959A938A93BA93AA93089577
:10254C0000240E160F060895552342F4503811F44A
:10255C00E0FF04C03196691F791F6BF050E85727D4
:10256C0011F45F93C8C05F3F31F0660F000C5795B4
:10257C006795752F08955F9300200AF0C7C0C0C0FF
:10258C0050E8192E1522880F991F9527550F8795FE
:10259C0050E8072E0522660F771F7527550F679594
:1025AC000895689401C0E8945F93F2DF703818F0D6
:1025BC007F3F08F4A0C056E1571BAAF45195583040
:1025CC000EF4593030F0EFEFFFEF6FEF7FE777F954
:1025DC001AC077275523B9F0EE0FFF1F661F771F20
:1025EC005A95D1F710C07727583028F0EF2FF62FD7
:1025FC00672F5850F9CF552331F076956795F7959D
:10260C00E7955A95D1F700200AF452DF5F910895AF
:10261C00689401C0E894309760407040B1F0002499
:10262C0026F0772312F4009443DF172E7EE111205D
:10263C0032F07A95EE0FFF1F661F111CF9CFEF2FAA
:10264C00F62F612D5F938ADF5F9108954F93AF0151
:10265C00FD01DA01AB01BC01CA01402D012C142E85
:10266C004F910895EA0FFB1F681F0895E095F095B0
:10267C006095EF5FFF4F6F4F08955F9381DF903848
:10268C0039F1703821F1572F591B2BF112F4DEDF81
:10269C00FACF583118F0AA27BB278827583028F0D2
:1026AC00AB2FB82F88275850F9CF552329F0869592
:1026BC00B795A7955A95D9F7502D512572F0D2DFC1
:1026CC0038F46795F795E795739513F41FC0BEDF43
:1026DC0045DF5F910895D8F7FBCFEA1BFB0B680B26
:1026EC0051F010F40094C2DF662392F3EE0FFF1F3B
:1026FC00661F7A95CBF7EE27FF27BF015F910895F0
:10270C00EFEFFFEF6FE77FEF5F910895EFEFFFEFD4
:10271C006FE77FE75F9108955F9332DF703859F36D
:10272C00903849F301240894791F23F424F30020F2
:10273C003AF3ECCF0F921F932F933F934F931127A4
:10274C0022279927689FA0018F9F302D410D591F7B
:10275C006B9F300D411D591F8E9F27D0BF9F25D0D9
:10276C006A9F23D0BE9F1DD0AF9F1BD0AE9F110D73
:10277C00291F391F491F591FE32FF42F652F522F83
:10278C004F913F912F911F910F9066232AF0550F77
:10279C00EE1FFF1F661F02C073954BF2D5DE5F91D3
:1027AC000895100D211D391F02C0200D311D491F28
:1027BC00591F08955F93E4DE703821F411200AF458
:1027CC009FCFA4CF903809F496CF01240894970B8F
:1027DC001BF4D4F30020F3CF792F1F932F933F9347
:1027EC004F931124112722273327A90190E2AE170A
:1027FC00BF078607410730F0AE1BBF0B860B410BA2
:10280C00089401C08894551F221F331F111CAA1F46
:10281C00BB1F881F441F9A9551F7F901612D4F91E9
:10282C003F912F911F91662332F0550FEE1FFF1F22
:10283C00661F7A954BF288DE5F91089599239AF082
:10284C00772342F0971748F029F4AE17BF07860795
:10285C0020F031F0989488940895989408940895F1
:10286C001894889408957723C2F7971798F3A9F7CB
:10287C00EA17FB07680788F399F3ECCF109639F049
:10288C00A8958DEC9AE00197F1F71197C9F7089587
:10289C00FFFFFFFFFFFFFFFFFFFFFFFFFFFFFFFF3C
:1028AC00FFFFFFFFFFFFFFFFFFFFFFFFFFFFFFFF2C
:1028BC00FFFFFFFFFFFFFFFFFFFFFFFFFFFFFFFF1C
:1028CC00FFFFFFFFFFFFFFFFFFFFFFFFFFFFFFFF0C
:10F9FC00FFFF9335FFFFFFFFFFFFFFFFFFFFFFFF41
:00000001FF
